:1089E20033302E3420202000003F0006005B004F71
:1089F2000066006D007D0007007F00670077007C45
:088A0200009300E500050000EF
:1071E80001230001250041066601C100C105C10255
:1071F800C104C101C10342064D00004106FE004121
:107208000710004106FA004106FB00012F00012487
:1072180000012A0041070C004406690000000044F0
:1072280006ED0000000041065A0044072500000052
:107238000041070A0041065900410723004206FCA5
:10724800000042070E000048072900000000000067
:10725800000041070102042B7FFFFFFF04260007FF
:1072680086A341070D00410643004806370400077E
:107278001D0CA7167E42063F000042064100004250
:107288000644000042064600004506480001020385
:1072980000420731000042072100004206FF0000BB
:1072A8004206670000460702303731363534410759
:0272B8000B00C9
:1057ED004F124AF09008A7E0FBA3E0FAA3E022F9DC
:1057FD00900007124A90C4540325E02429F582E451
:10580D003407F583E0FEA3E0FF7C047D00124E9586
:10581D009008D4124E269008D4E0FCA3E0FDA3E03E
:10582D00FEA3E0FFE47BE87A03F9F8124CF190084F
:10583D00D4124E269008D4E47FFF7EFFFDFCE0F8E5
:10584D00A3E0F9A3E0FAA3E022F9900008124A9030
:10585D00C4135401FFE52FFD3395E0FC74112DF5B4
:10586D008274073CF583EFF0E92408F9E43AFA0273
:10587D004A779009ABE0FCA3E0FDA3E0FEA3E0FFB7
:10588D00E4F9F8124C669009AB124E269009ABE084
:10589D00FCA3E0FDA3E0FEA3E022AF2FEF3395E0E4
:1058AD00FE7C007D0B124B24746B2FF974043EFAB1
:1058BD002290089D7B017A08798AEBF0A3EAF0A388
:1058CD00E9F022AF2FEF3395E0FEEF25E0FFEE3349
:1058DD00FE2274452FF58274043EF583A3E0C4F8CF
:1058ED00540FC868FF058222F9900008024A90F90A
:1058FD00900007124A901313540325E02429F582D2
:10590D00E43407F583E0FEA3E0FF22900007F912CF
:10591D004A90131313540722FF2473F58274063E25
:10592D00F583EDF074732FF58274063EF583E0FF79
:10593D0090047075F00BEB124E63EA75F00BA42515
:10594D0083F58322F9900009124A90C31354032260
:10595D009009A87C007D05E0FEA3E0FF024B36E434
:10596D00FFFEFDFCD3AB2EAA2DA92CA82B024D902A
:10597D00FDE0FAA3E0FB25E0FFEA33FE74992FF575
:10598D008274073EF583ECF0A3EDF0229000051232
:10599D004A90FF900006124A90FD900004024A9032
:1059AD00900002F9124BE2FFAEF022F990000712BF
:1059BD004A90540722900002F9EE8FF0024C39E024
:1059CD00FF75F00A124A5590090FF0EF75F00A02B3
:1059DD004A559008E4E0FEA3E0FFC322124C668F07
:1059ED00298E288D278C2622FF131313541FFEEFAB
:1059FD0054C7FFEE045407FE33333354F84F024AB5
:105A0D00F0E0FEA3E0FFE4FCFD22EB5FFFEA5EFEAB
:105A1D00E95DFDE85CFC229008E4E0FCA3E0FD25D7
:105A2D00E0FFEC33FE229009A1A3A3E0FEEE22F9E4
:105A3D0090000A124A90540722AF23EF3395E0FEEF
:105A4D00EF7803221582E0C454F048229009AB127E
:105A5D004E26E47FFF7EFFFDFC22F9F8124C669086
:105A6D000866124E2690086622AF2FEF3395E0FEA2
:105A7D0074112FF58274073EF583E05401C433543D
:105A8D00E0FF22F9900006024A902474F582740614
:105A9D003EF583E022E52E9529F52EE52D9528F589
:105AAD002DE52C9527F52CE52B9526F52B22900829
:105ABD00AAEEF0A3EFF0D3E49FE49E22F9124BB7C8
:105ACD00FFAEF022F9900009024A909008E4A3E09D
:105ADD00FF74017E00A80708229008E4E0FEA3E011
:105AED0090047275F00B124E63EE22EF9408EE6483
:105AFD0080948022FFED64015401FE22EF3395E086
:105B0D009008E4F0A3EFF022FFE47BE87A03F9F8C4
:105B1D00024CF19009A1A3A3A3E022900003024A35
:105B2D0090AF29AE28AD27AC2622900659E0FFD3C1
:105B3D006480F82290091174FFF0900910F090091B
:105B4D000FF090090EF0229008CDE0C4F8540FC864
:105B5D006822E0FFD364809480900934222401FFF1
:105B6D00E43EFEE43DFDE43CFC22900666E064016B
:105B7D00229008AAE0FEC3EE22246DF974063EFAC7
:105B8D007401229008E4124E269008E422F9900048
:105B9D0007024A909008D4A3A3E0FEA3E0FF229051
:105BAD0008E5E094049008E4E064809480223EF5DA
:105BBD0083E0F59BE4FFFE2274452FF58274043ECD
:105BCD00229008E5E025E0FF9008E4E033FE229006
:105BDD0008CCE0C454F04822900644E0FEA3E0FF58
:105BED0022FDE52FFB3395E0FAEBAE027803229010
:105BFD0009ABA3A3E0FFA3E09009A8CF22E0FFA388
:105C0D00E09006F1CFF0A3EFF022E0FFA3E09006C5
:105C1D00F3CFF0A3EFF022E0FFA3E09006F5CFF075
:105C2D00A3EFF022900404E0540722FFE4F0A3EF69
:105C3D00F022752EFF752DFF752CFF752B7F223EE3
:105C4D00F583E01313540322EF3395E0FEEF24EBBD
:105C5D00FFEE34FF229008E4E0FCA3E0540725E0BA
:105C6D00FF2253A0F743A0102243A00853A0EF2218
:105C7D0090090EAFF0EFF0A3E02290090F74FFF042
:105C8D0090090E740AF022D3EF648094802274B9C7
:105C9D002FF58274072274FFF52EF52DF52C752B3B
:105CAD007F22FFEE3395E0FDFC229008CCE0FCA3B3
:105CBD00E02274052FF58274042274252FF5827469
:105CCD000422F9EE8FF0024C1AE4900900024E26E0
:105CDD00E05438FF9009A522E05407FF9009A52252
:105CED001313135401FDEF22F9900001024A90FDA8
:105CFD00900005024A9074292FF58274073EF583B2
:105D0D0022FFEE3AFEED39FDEC38FC22F4FFEEF405
:105D1D00FE3395E0FDFC225438FFE054C72275BCDC
:105D2D00F990070122900870024E26FFEEF0A3EFC6
:105D3D00F022FBEDAE047803227B017A09790E2265
:06503300E4900723F022C7
:075005009007237401F02263
:10503C0075FFDE75FFADE4F5E6F5E7C2AF128C98AF
:10504C00900724EFF090066D125C0A90066F125CCC
:10505C0017900671125C24E4A3F0A3F0A3F0F5847E
:0E506C00127AE21286CB128B60128595E4FF59
:10507A0075F002EFA42405F582E5F03404F583E027
:10508A00FDA3E09008A6CDF0A3EDF09008A6E0FC01
:10509A00A3E0FDEF25E02499F582E4340712599143
:0D50AA00EF25E02433F582E434071259911C
:0A50B7000FEFB433BED2AF128CAD80
:1050C1007F407E0D7D037C0090063312584BFBC35D
:1050D100124DA6500F90063312589C125B6A90062F
:1050E10033124E261285449008A6EFF07003025643
:0150F1006559
:1050F2001258A7A374011258C89008A6E014B41657
:1051020000400302566590511675F003A4C583252D
:10511200F0C583730251580251AC0251DA0251E0D8
:105122000251E602521E0252C70253EE0253F80225
:1051320054590254790254D70255380255AE0255D9
:10514200CA0255E702560202562502565802565D19
:10515200025662025648E52570030256651257F15F
:1051620012595164036031125875FFC4135401FD82
:10517200EF54DF125B01C43354E01257ED1258F5BD
:10518200C4135401FFE52FFD3395E0FC74112DF596
:105192008274073CF583EFF01257F11258F5542050
:1051A200FF900663E054DF025455E5257003025672
:1051B200651257F1125876FFC4125CEE54BF125BAF
:1051C20001C4333354C01257ED1258F55440FF90C6
:1051D2000663E054BF025455128ADF025665128DEF
:1051E20095025665E52570030256651257F1240AA9
:1051F2001258781259F5EEC39405400D1257F12456
:105202000A12587854C7124AF01257F1F990000A5C
:10521200124A90900665125D24025455E5257003EA
:105222000256651257F11259B8600BE92407125859
:065232007854F80252B4AA
:105238001258D074D92FF58274073E125910125A99
:10524800BB501AC3E094999008AAE09401500E123A
:1052580057F1240712587854F84401804F9008AA4F
:10526800E0FEA3E0C39499EE94014013EE94085035
:105278000E1257F1240712587854F84402802D90E2
:1052880008AA1259E2EE94084016EF9465EE940EBF
:10529800500E1257F1240712587854F84403800C22
:0F52A8001257F1240712587854F84404124AF0B0
:1052B7001257F11259B8FF900662E054F80254559C
:1052C700E5257003025665125B7760030253671288
:1052D70057F1125918600BE9240712587854C7027E
:0252E70053531F
:1052E9001258D074992FF58274073E125910125A28
:1052F900BB5017C39008AAE09440500E1257F124EE
:105309000712587854C744088040125B7E94404085
:1053190013EE9480500E1257F1240712587854C78F
:1053290044108026125B7E94804013EE94C0500E88
:105339001257F1240712587854C74418800C125791
:0D534900F1240712587854C74420124AF08E
:105356001257F1125B9A900662125D244FF00256C4
:10536600001257F11258F55407600812587554F890
:035376000253D708
:105379001258D0125C9B3E125910125ABB5015C3D9
:105389009008AAE09440500C1257F112587654F83C
:105399004401803A125B7E94404011EE9480500C97
:1053A9001257F112587654F844028022125B7E9407
:1053B900804011EE94C0500C1257F112587654F8EF
:1053C9004403800A1257F112587654F84404124AD9
:0153D900F0E3
:1053DA001257F11258F55407FF900663E054F84F3C
:1053EA00F0025600900403E06401F0025665E525D8
:1053FA0070030256651257F12409125878FFC31335
:10540A00FEEF54F9FFEE045403FE25E04F124AF072
:10541A00EE6403700A1257F11258564420801A1289
:10542A0057F11259517015125A7612587554DF12E3
:10543A0057ED240912587854F9124AF01257F1120A
:10544A005AD15406FF900664E054F94F0255E4908D
:10545A000666E0FFC374039FFFF0BF01059006696B
:10546A0080039006ED124E32FFFFFFFF025665E5FC
:10547A00257003025665125B779008A770271257AA
:10548A00F4125876FF125CED54F7125B0133333392
:10549A0054F81257ED1258F55408FF900663E05479
:1054AA00F74FF080251257F4125876FFC45401FDC5
:1054BA00EF54EF125B01C454F01257ED1258F55431
:1054CA0010FF900663E054EF4FF0025600E5257096
:1054DA0003025665125B779008A770291257F412D7
:1054EA005876FFC4125CED547F125B01C433333328
:1054FA0054801257ED1258F55480FF900663E05419
:10550A007F4FF080261257F42409125878FF54016D
:10551A00FDEF54FEFFED640154011257ED125AD10A
:10552A005401FF900664E054FE4FF0025600E52550
:10553A007003025665125B7770311257F124091213
:10554A0058781259F5EED39406400D1257F12409F2
:10555A0012587854C7124AF01257F1125AD15438D5
:10556A00FF900664E054C74FF080371257F1240ABF
:10557A00125878FF54F8FEEF045407FF4E124AF00F
:10558A00EFC39407400D1257F1240A12587854F8C1
:10559A00124AF01257F1125A3CFF900665E054F88D
:1055AA004FF08052E52570030256651257F1F91241
:1055BA004A7764011257EEF9124A7790065B801A0D
:1055CA00E52570030256651257F1240112587864D2
:1055DA00011257EE125CF590065CF0802E900404DE
:1055EA00E0FF54F8FEEF045407FD4EF0EDC39403B8
:1055FA004004E054F8F08013E525601490065AE060
:10560A0004F0C3648094834002E4F0128934804B2E
:10561A0075250190065A7401F0804020000EE4902E
:10562A000402F0128DB7C205C204802FA202B392FF
:10563A0002300206C20BD2048021C204801D9007E8
:10564A0024E0FF7BFF7A8979E212849A800D632530
:0B565A00018008127E5A8003127EF7C8
:1056650030030E900723E07006A3E0FF128C38C2CA
:10567500037B017A08798A12898EEF70030250C183
:1056850090088CE0124E6F56E904570A0556B91476
:1056950056AB1656B21756BE1A56D21B56DD1D56B8
:1056A500E31E00005734D202D204025734C202C2AC
:1056B50004025734D20002573490089A1258C11286
:1056C5004A77FE900724E0FF6E70648005900724FA
:1056D500E0FF128C810257341250050257341250E4
:1056E500330257341258BE125B28FF900724E06F2F
:1056F500703D30023290089D041258C8125999FB2A
:1057050012819A80221258BE125B28FF900724E06E
:105715006F701C30021190089D041258C8125999D7
:10572500FB127F91128595900724E0FF128C512082
:10573500020302567690088CE01460381460202429
:10574500FB604614607124F960030256767B017A8A
:1057550008798A9008A31258C7128B000256761250
:1057650057D990089A1258C7125B28900402F01274
:105775008DB7803D1257D990089A1258C7125B28E9
:10578500900402F012859580281257E39008A01224
:1057950058C7125B28FF1259A7125CFCFBC0039087
:1057A50008A01257F4125A9090092AF0D003127DDE
:1057B5001C128D6B0256761257E39008A01258C73B
:1057C500125B28FF1259A7125CFCFB1270A9128DFF
:0457D5006B02567697
:1057D900128CE57B017A08798A22128CE57B017AA1
:0457E90008798A228F
:108C980030B60930B7037F41227F422230B7037FC5
:058CA80061227F622241
:107AE20090099EE584F075FFDE75FFAD75840F7514
:057AF2009601758C20D7
:107AF700E4A3F0A3F090099F125A0E7B407A9CF9F9
:107B0700F8D3124D9040109009A0E004F070E69071
:077B1700099FE004F080DE8D
:107B1E00E4F58475EF0675840F758A83F597758481
:107B2E000F758904F58475B73075840F4389017517
:107B3E008D01758F01758E0490099A124E320000D8
:107B4E000000E4FF7E01FDFC90099A12584BFBC326
:107B5E00124DA6501190099A12589C125B6A900908
:107B6E009A124E2680DC438902E58920E4129009A0
:107B7E009A124DF1E4FB7A01F9F8C3124DA650E9C1
:107B8E00759702E4F58A90099EE0F584E4F5841277
:107B9E0089BA128BB7128CF6900724E0FF128D462D
:107BAE0043F602128D81128D061287DE90099A021B
:027BBE004E2651
:1089BA0075840F75A4CF75A71C75B0E7E4F5E27549
:1089CA00A6FF75E10375E3C0F5A57590FF75ADE3E4
:0889DA0075AD63F5A5F58422DB
:108BB700E4F58443E60875DA3175DB3175DC317528
:0A8BC700DD3175D983D2DEF584227A
:108CF600D2AF759A4075F809759D01C286C2872262
:0A8D810075E8C075BCF875D1032237
:108CD300E4FDFCC3ED9FEC9E50070DBD00010C802D
:018CE300F29E
:018CE400226D
:108D060075840275E88075BCF975D103E4F5842293
:1087DE00AB84E4F584F588758DF0F58B758910F50D
:1087EE008E7588409009DA124E320000F00DE4F5D5
:1087FE008475CC0D75CDF075CA0D75CBF0F5C975B8
:10880E00C80443A828AF038F849009DA12589CFF3E
:01881E002237
:108CAD00E4F5BB758402900701E0F5BBE4F5844360
:038CBD00E7122299
:108ADF00AF231258A97B01900404E04408F09000E2
:108AEF000A12591CFF6003BF0406127DBD125CA35E
:018AFF002254
:088D9500900404E054F7F02201
:107DBD00125A91543FFF7005E5230480071259A70D
:107DCD007009EF149009DEF0027E45125A46C33356
:107DDD00CE33CED8F9FDAC062473F58274063CF58E
:107DED0083E0D3648094804019125A91543F1490CB
:107DFD0009DEF074732DF58274063CF583E014F002
:027E0D008036BD
:107E0F00AF231258A97B019009DF1258C7E523044D
:107E1F009009DEF01259A7900005124B02125CFD7B
:107E2F00FD125A46C333CE33CED8F92473F582747C
:067E3F00063EF583EDF0A4
:107E45009009DEE0C3648094904002E4F09009DE7E
:057E5500E0FF0288CCF3
:1088CC00E490070CF08523248F239006F704F0A383
:1088DC00F0A3F0EF3395E0FE90047575F00BEF12FA
:1088EC004E63EE125948E01313135407FFBF0403F1
:0488FC00128D952222
:108CC000125C31FFBF010B90070DE0FF1288CC1240
:038CD0005CA32280
:03503900025D4DC8
:105D4D00C0E0C0F0C083C082C0D075D000C000C01C
:0D5D5D0001C002C003C004C005C006C0079D
:105D6A00758402C2ED900861E5BEF0900701E02457
:105D7A00FD7003025E081470030261DA24FD7003E9
:105D8A000261F924056003026255900861E09007F8
:105D9A00FD125C387D327F32126DE290070DE09081
:105DAA000643F09006FCE0C4540FFD900469E0C479
:105DBA00F854F0C8A3E0C4540F482D90070DF0D34F
:105DCA00940F4004E024F0F0900643E0FE90070DA3
:105DDA00E0FFB506046523600D125C31FEBE0206C3
:105DEA001288CC125C3F900643E0FF90070DE06FEB
:0E5DFA006003128934125D2B7403F0026255AF
:105E080090070E125A0E900878124E2690087E12AD
:105E18004E3200000163900882124E3200071C00C7
:105E2800AF231258A97B019008861258C7E523FDB5
:105E38003395E0FCED125A2C1258DFD582021583F7
:0F5E4800125A5190086CF0A3EFF01259B9602D67
:105E5700EDAE047803C333CE33CED8F9125A97C4C4
:105E67005403FF900889F01258D3125D03E0C4F879
:0B5E770054F0C868FFA3E0C4540F48BB
:105E8200800EAF231258D2125BC5F583E0FFA3E068
:105E920090086ECFF0A3EFF090086EE0FCA3E0FD57
:105EA200EC1313543F900865F0EC5403FEAF05E485
:105EB200FCFDA3125A6F12589CFFE47B637A011215
:105EC2005A6712584BFBC3E49BFF74A89AFE740CEA
:105ED20099FDE498FC900866124E26900865E0252C
:105EE200E02437F582E43406125910900862EEF08D
:105EF200A3EFF0FBAA06E4F9F890086612589CFF9B
:105F0200124CF1125D329006FEE4F09008861257B0
:105F1200F41258F5C413540720E0030260671259C3
:105F22005264036003025FAB1258D0125BC5125970
:105F320010C39416EE9401500AEF94A4EE9400401C
:105F420002805DC3EF94FFEE9402500AEF94B9EE23
:105F520094024002804AC3EF94A7EE9406500AEFDF
:105F620094F8EE940540028037C3EF94EBEE940868
:105F7200500AEF9495EE940840028024C3EF9417E0
:105F8200EE940C500AEF94D1EE940B40028011C3B0
:105F9200EF945BEE940F500EEF94E9EE940E4006F0
:105FA2009006FE7401F0026067E47FC77E01FDFC8B
:105FB20090087012584BFBD3124D90400C9008740D
:105FC200124E32000002808045E4FF7E01FDFC900B
:105FD200087012584BFBD3124D90400C900874126B
:105FE2004E32000001408026E47F8FFEFDFC9008C7
:105FF2007012584BFBD3124D909008744009124E08
:1060020032000000A08007124E32000000509008BB
:106012006CE0131313541F7E00125D38C3941CEE00
:10602200940050047F0180027F0090086CE0FCA382
:10603200E0FDD39404EC940040047E0180027E00D3
:10604200EE5F602C7E00ED540790086C125D3864A0
:1060520007600A90086CE07002A3E070139006FEDD
:106062007401F0800B90087012589CFFA3124E2608
:106072007FA37E867D077C0090087412584BFB122A
:1060820059E97808124DCA1259EC9008861257F451
:10609200125951601024FD600C24027014125B2E00
:1060A200E47B088006125B2EE47B40FAF9F8125971
:1060B200E9900861E09007F9125C387D307F301278
:1060C2006DE2900864E0FF900708E4F0A3EFF0901F
:1060D2000465A3E0900864F0900467E0FFA3E090F9
:1060E200087CCFF0A3EFF0E02480F090087CE0344D
:1060F200FFF0E0FEA3E0125CAF90087812584BFB71
:10610200124C66125D3290087012589CFF780F1282
:106112004DCA125D32900864E0FFE4FCFDFE900877
:106122007012584B2F125D0EA3124E26E47FFFFE13
:10613200FDFC90087412584BFBD3124D90400A900C
:106142000874124E32000000FF90087412589CFF2F
:10615200EC33500A900874124E320000000090088E
:1061620074A3A3A3E0900864F0E0FFC413135403E4
:10617200A3F0EF543FFFE4FCFDFEA3125A6F125846
:106182009CFFE47B08FA125A6712584BFBC374F85F
:106192009BFF74039AFEE499FDE498FC125A6C1278
:1061A200589CFF900865E0F9F8124DB790086AEE26
:1061B200F0A3EFF0125B2E7808124DCA1259ECAB25
:1061C20029AA28A927A82690086A125A0E1259E964
:0861D200125D2B7404F0807BC8
:1061DA00900861E0FF9007FBE4F0A3EFF07D317FC8
:0F61EA0031126DE275BCF89007017407F0805C0C
:1061F90090063FE0FEA3E0FFA3EEF0A3EFF09008C6
:1062090061E0FD90063FE4F0A3EDF0D3EF9480EE5A
:106219009400500EE0948090063FE09400400312F1
:106229008ADFD3900640E0942590063FE094005021
:1062390008E50B5404FFEF70089007107401F08013
:0C62490005900710E4F0125D2B7402F0C9
:0C625500900701E0F5BB75840043E810E1
:10626100D007D006D005D004D003D002D001D00091
:0B627100D0D0D082D083D0F0D0E0323B
:0350300002409AA1
:10409A00C0E0C0F0C083C082C0D075D000C000C0EC
:0D40AA0001C002C003C004C005C006C0076D
:1040B700AF231258A99008D874011258C8AF24EF3B
:1040C7003395E0FE1258B2A374011258C8125A462B
:1040D700C333CE33CED8F99008DE125B861258C8A8
:1040E700AF24125A48C333CE33CED8F99008E11221
:1040F7005B861258C8C2EDE4FFFEFDFC900725124F
:10410700584BFBD3124D90401D90072512589CFF2A
:10411700EF24FFFFEE34FFFEED34FFFDEC34FFFC30
:10412700900725124E26E47F01FEFDFC900725121D
:10413700584BFBC3124D90700D128CC0900725127F
:104147004E3200000000AFBFEFFFADBEED9008CCD0
:10415700CFF0A3EFF0125B3774809840030242E17F
:0B416700C3EF6480949040030242E12B
:10417200125B09125B77707B125CB79008E41259EC
:104182007DAF03125ADE8005C333CE33CED8F91287
:104192005CAF90066912584B125A184D4E4F604B45
:1041A200125BCE74992FF58274073EF583E0FCA36F
:1041B200E0FD74332FF5827407125990900669124C
:1041C200584BFBC000C001C002C003125AD8800580
:1041D200C333CE33CED8F9125D19D003D002D00149
:1041E200D000125A17900669124E269008E4A3E0F6
:1041F20002427A125CB7FD9008E4E0FAA3E0FB25E4
:10420200E0FFEA33FE125C9B125990AF03125ADEB2
:104212008005C333CE33CED8F9125CAF9006ED12CF
:10422200584B125A184D4E4F6047125BCE125C9B90
:104232003EF583E0FCA3E0FD74532FF58274071270
:1042420059909006ED12584BFBC000C001C002C04D
:1042520003125AD88005C333CE33CED8F9125D1972
:10426200D003D002D001D000125A179006ED124EA0
:10427200269008E4A3E02410FDFF126DE2125AE634
:10428200125948E01313135407601A125A24125C8D
:10429200BF125C4C125D3FC333CE33CED8F9125AF3
:1042A2009754FC4BF09008E4E0FEA3E090047312F4
:1042B2005AF0125948E0540770030243E4125A2498
:1042C200125CC7125C4CFF25E025E0125D3FC33350
:0C42D200CE33CED8F9125A9754F34BF0BB
:0B42DE000243E4900659E064107038C1
:1042E900125B54FF125BDCFEE4FCFD125B9012587A
:1042F9009CFFE4FB7A04F9F8124C66125B901258A1
:104309009C125B15125B90A3A3E0FFA3E09006FC4F
:05431900CFF0A3EFF05E
:10431E000243E4125B377411648098500EC3EF644D
:05432E0080949550068B
:03433300EF24EF85
:104336000243CA125B3774156480985054C3EF6405
:054346008094A5504C1D
:10434B00125C55FE125B0D2420FFE43EA3F0A3EF9D
:10435B00F0125CB79008E612597DAD03AF05126DF4
:10436B00E2125AE6125948E05407606D125A2412B1
:10437B005BC5125C4DFFC454F0125D3FC333CE33AB
:0A438B00CED8F9125A9754CF4BF028
:10439500804D900659E0FDB42510125B54FE125B6A
:1043A500DC90070EF0A3CEF08035D3ED6480F87471
:1043B500266480985029900659E0FFC3648094AA2A
:0243C500501D89
:1043C700EF24DAFF9008E4F0FD125B54FB125BDC8C
:0D43D700FAED1258D3125D03EAF0A3EBF0EB
:1043E4009008D81257F41259186028900403E0700A
:1043F400429008DE1257F4125B9A1259059008D8BD
:104404001257F490000912591B12494B1257F4F930
:10441400EE801BAF231258D2125CBF1258E6D5822D
:10442400021583125A51F99008DE1257F4C98FF01D
:10443400124C1A9008DB1257F41259186029900490
:1044440003E070439008E11257F4125B9A12590585
:104454009008DB1257F4F990000912591C124955BF
:104464001257F4F9EE801BAF241258D2125CBF121B
:1044740058E6D582021583125A51F99008E1125771
:10448400F4C98FF0124C1A9008D81257F41258F548
:1044940054076020900403E070379008DE1257F44C
:1044A4001258FC9008D81257F4125A3CFDAB231250
:1044B40076B28014AF231258D2125CC71258E6D5D4
:1044C40082021583125A51FE9008DE1257F41259D3
:1044D400C29008DB1257F41258F554076020900478
:1044E40003E070379008E11257F41258FC9008DB8F
:1044F4001257F4125A3CFDAB241276B28014AF2446
:104504001258D2125CC71258E6D582021583125A89
:1045140051FE9008E11257F41259C29008D812576C
:10452400F41259B86025900403E0703C9008DE1240
:1045340057F41257FCFBD3124DA6400A9008D4122C
:104544004E320000FFFF125BA18011AF231258D23C
:104554001258DFD582021583125A51FE9008DE12DA
:1045640057F49000041259C59008DB1257F41259FD
:10457400B86025900403E0703D9008E11257F412EE
:1045840057FCFBD3124DA6400A9008D4124E3200B9
:1045940000FFFF125BA18011AF241258D21258DF22
:1045A400D582021583125A51FE9008E11257F4F98C
:1045B4009000041259C69008D81257F41259187072
:1045C4001F9008DE1257F4125AC99008D81257F4F3
:1045D400F990000912591C12494B1257F4125CCF7E
:1045E4009008D81257F41258F5540770219008DE39
:1045F4001257F41259AD9008D81257F4125A3CFDD0
:10460400AB231276B29008DE1257F41259C2900608
:10461400FAE4F09008D81257F41258F5131313540F
:104624001F30E0269008DE1257F4125AC91286355C
:104634009006FAEFF09008DE1257F4125AC9128667
:10464400839008DE1257F4125CCF9006FBE4F090DE
:1046540008D81257F41258F5C4540F30E0269008C5
:10466400DE1257F41259AD1286359006FBEFF09026
:1046740008DE1257F41259AD1286839008DE1257E1
:10468400F41259C29008D81257F41258F5C41313EF
:1046940013540130E0509008E11257F4125AC990B3
:1046A40008DB1257F4F990000912591C12495512EB
:1046B40057F4125CCF9008DE1257F4125AC9E4FC86
:1046C400FDC004C005C006C0079008E11257F412EB
:1046D4005AC9125CD6D007D006D005D0041283691B
:1046E4009008CEEE80109008DE1257F4F9124BB702
:1046F400FF9008CEE5F0F0A3EFF09008D81257F43D
:10470400125AD130E0529008E11257F41259AD9088
:1047140008DB1257F4125A3CFDAB241276B290080F
:10472400E11257F41259C29008DE1257F41259AD2F
:10473400E4FCFDC004C005C006C0079008E11257A0
:10474400F41259AD125CD6D007D006D005D00412AD
:1047540083699008D0EE80139008DE1257F4F99024
:104764000002124BE2FF9008D0E5F0F0A3EFF090C6
:1047740008D81257F41258F5C4131354039008DEE2
:1047840030E0351257F49000041259B0E4FCFDC037
:1047940004C005C006C0079008E11257F4F9900060
:1047A400041259B1125CD6D007D006D005D0041239
:1047B40083699008D2EE80101257F4F99000041225
:1047C4004BE2FF9008D2E5F0F0A3EFF09008CE1290
:1047D4005C0A9008D0125C179008D2125C249007EF
:1047E4000A125B3A748098505DC3EF6480949050D1
:0147F400556F
:1047F500125B09125C62A3EFF0C3EC648094804005
:104805000A125BAC5005125C6F80141259DF9404D8
:10481500EE64809480400E125AF85009125C767549
:10482500BB000248DD1259DF125AF9400FEF940C14
:10483500EE648094805005125C6F8003125C76757F
:02484500BB01B5
:104847000248DD90070AE0FFB4100675BB02024973
:1048570017EFB411030248F9EFB41203024902EF4C
:10486700B4130302490BEFB41403024914D3EF64E2
:1048770080F874156480985068C3EF648094A550DD
:0148870060D0
:10488800125C55125B0D125C62EF04A3F0C3EC647A
:10489800809480400A125BAC5005125C6F80141241
:1048A80059DF9404EE64809480400D125AF8500841
:1048B800125C7675BB00801D1259DF125AF9400F41
:1048C800EF940CEE648094805005125C6F800312A4
:0E48D8005C7675BB0153A0F89008E6E042A0A4
:1048E600802F90070AE0FFB4250575BB038022EFF1
:1048F600B4260575BB048019EFB4270575BB058082
:1049060010EFB4280575BB068007EFB4290375BB05
:104916000790070AE0900659F090070A04F0C3646E
:0A4926008094AA4002E4F0126AB87F
:10493000D007D006D005D004D003D002D001D000DB
:10494000D0D0D082D083D0F0D0E032FDAB2312762D
:0F495000B29008DE22FDAB241276B29008E1226D
:108A5500EF252FF52FD36480948F4003E4F52FC3C2
:108A6500E52F648094805003752F0FE52560031270
:038A750068C122B3
:1068C100AF0BAE0AAD09AC08124D839009A1124E6F
:1068D100261258A79009A574011258C8125B2054BA
:1068E10001FFEF6016900663E05420FF9009A512A6
:1068F10057F412587654DF4F124AF0125B205402BB
:10690100FFEF6016900663E05440FF9009A512570F
:10691100F412587654BF4F124AF0125A335401FE02
:10692100EE604A900664E0C31354036403700D9053
:1069310009A51257F4125856442080169009A51241
:1069410057F4125951FFBF030C125A76125875545D
:10695100DF4F124AF0900664E05406FF9009A51239
:1069610057F4240912587854F94F124AF0125A3345
:106971005404FEEE602E900666E0900663B40111A9
:10698100E05408FF9009A51257F412587654F78085
:106991000FE05410FF9009A51257F412587654EFE6
:1069A1004F124AF0125A335408FEEE6033900666D5
:1069B100E0B40114900663E05480FF9009A51257DA
:1069C100F4125876547F8014900664E05401FF90CD
:1069D10009A51257F4240912587854FE4F124AF0AF
:1069E100125A335410FEEE602D900666E0B4011287
:1069F100900664125CDD1257F4240912587854C7CA
:106A01008010900665125CE51257F4240A1258783A
:106A110054F84F124AF0125A335420FEEE6010908F
:106A2100065BE0FF9009A51257F4F9EF124AF01244
:106A31005A335440FEEE601390065CE0FF9009A5C6
:106A41001257F4F9900001EF124B02125B205440EF
:106A5100FFEF602B900666E0B40112900662125CB3
:106A6100DD1257F4240712587854C7800E9006633C
:106A7100125CE51257F412587654F84F124AF0128C
:106A81005B205420FFEF6011900662125CE5125703
:106A9100F42407125878125A08125B205410FFEFA1
:106AA1006014900665125CDD1257F4240A125878BE
:066AB10054C74F124AF029
:016AB70022BC
:054EEE009009C0EDF089
:104EF300900646E475F001124B8BFED3E5F0125A8F
:104F0300F9401EE4900646F0A3F090064475F001C4
:104F1300124B8BFEE5F064044E7006900644F0A33A
:104F2300F0125BE564034E6006EF64014E7022905D
:104F33000646E0FEA3E0FF4E7009900646F0A30488
:104F4300F0800EEF64034E7008900646F0A37407DA
:104F5300F0125BE52404FD7401A805088002C33345
:104F6300D8FC900654F0C3900647E0940890064698
:074F7300E0648094805059B6
:104F7A008F828E83124A90FF9009C2F01258D3741E
:104F8A00EA2FF58274893EF583E493FC740193FD5C
:104F9A00900646A3E0FB74017E00A803088005C3BF
:104FAA0033CE33CED8F9FFEC5EFEED5F4E6008904B
:104FBA000654E02BF08005E4900654F09009C2E014
:074FCA00C3648094805033A2
:104FD100802C125BE5EE702BEF14600A1460111443
:104FE100600E2403701D9009C1E060028008800EEC
:104FF1009009C0E06008900654E02407F022E49094
:035001000654F062
:015004002289
:077EF700E5257003027F8BFB
:107EFE001258A7900A0A74011258C890065AE064E4
:107F0E00017028900A0A1257F4125A90543FD394D3
:107F1E00004012E92406125878FF54C0FEEF1454A4
:107F2E003F4E124AF0128934027F8890065AE0645E
:107F3E00027042900A0A1257F4F91259A7FFD3643D
:107F4E00809481400A90000474FF124ABD800BEFAA
:107F5E0070089000047413124B02900A0A1257F420
:107F6E00F91259A7125BEEC333CE33CED8F912599C
:0D7F7E0025EFF080057FFF128A550289343F
:067F8B007FFF128A55225F
:077E5A00E5257003027EF133
:107E61001258A7900A0D74011258C890065AE0647E
:107E7100017025900A0D1257F4125A90543FC39481
:107E8100105012E92406125878FF54C0FEEF045432
:107E91003F4E124AF0027EE490065AE064027048B6
:107EA100900A0D1257F4F91259A7FFC364809493F5
:107EB100500DEF600A9000047401124ABD800BEF6F
:107EC100B41307900004E4124B02900A0D1257F408
:107ED100F91259A7125BEEC333CE33CED8F912593A
:107EE10025EFF012893480057F01128A5502893409
:067EF1007F01128A5522F8
:03501200028D53B9
:0C8D5300C2CF75840243E8107584003222
:106C5200900666E0B401079006FAE0FC8005900613
:106C6200FBE0FC125952FF6403601590064FE0FEF0
:106C72007401A807088002C333D8FC4E90064FF077
:106C8200900652E0FF124A77FEEF4E900652F0E075
:106C9200FF125CF625E0FEEF4E900652F01258F617
:106CA200FEC413540730E0139006FEE090064F60D6
:106CB20006E04410F08004E04420F090064FE0FF2C
:106CC200EEC41313540133333354F8FEEF4EF090F5
:106CD2000666E0900650B4010BE0FF1258F6C413AA
:106CE20013138005E0FF125AD25401FEEF4E9006B4
:106CF20050F0900666E0FF640170131258F6131309
:106D020013541F30E021EC9006506017800F125888
:106D1200F6C4540F30E010EC9006506006E04402D6
:106D2200F08004E04404F0EFB40108125AD21313C5
:106D320013800690000A124A905407FDEDB405092B
:106D4200900651E04420F0803EED7009900651E03B
:106D52004401F08032EDB40109900651E04402F0A2
:106D62008025EDB40209900651E04404F08018ED4C
:106D7200B40309900651E04408F0800BEDB4040717
:106D8200900651E04410F090000A12591CFF602155
:106D9200900653E0FE74482FF582E43406F583E052
:106DA200FF7401A807088002C333D8FC4E90065333
:016DB200F0F0
:106DB300125B9BFF54076007900653E04410F0906A
:106DC3000666E0B4010AEF1313135407601080073B
:0E6DD3001258F654076007900653E04420F073
:016DE100228F
:1078D200E49009D8F0A3F09009D81259E29405EE89
:1078E20064809480501C744F2FF58274063EF58399
:1078F200E4F09009D9E004F070DD9009D8E004F0DA
:1079020080D5E5256004AF2F8002AF231258A990DD
:1079120009D574011258C89009D51257F4F9126C9E
:1079220052125C31FDBD0109900652E04404F08020
:107932000ABD0207900652E04408F0900650E0FFAC
:10794200900666E033333354F8FEEF4E900650F063
:10795200300407900652E04410F0900652E0FFE532
:1079620025C43354E0FEEF4EF0900404E0131313E9
:10797200541F90064F30E006E04480F08004E0445B
:1079820040F0900653E0FF900403E0C4333354C048
:10799200FEEF4E900653F0C2FA9009D8E4F0A374B9
:1079A20004F053F87FE59A20E7FB9009D8E0FEA3A4
:1079B200E0244FF5827406125BBB0FBF00010EEF8D
:1079C20064324E70F59009D9E024FFF09009D8E0B6
:0E79D20034FFF0E0B4FFCBA3E0B4FFC6D2FA5E
:0179E0002284
:106AB800E490090CF0A3F090090C1259E29403EE4B
:106AC80064809480501C74542FF58274063EF583BC
:106AD800E4F090090DE004F070DD90090CE004F09A
:106AE80080D5E52330E31C900656E0FFE5235407E4
:106AF800FE7401A806088002C333D8FC4F900656DE
:106B0800F08017900655E0FFAE237401A8060880B0
:0C6B180002C333D8FC4F900655F0C28732
:106B24001258A790091274011258C8AF2F125A486C
:106B3400C333CE33CED8F9246DF974063EFA9009E6
:106B44001574011258C89009121257F4125A90542D
:106B54003FFF900918F01259A7900919F0900915F0
:106B64001257F4125A9090091A1259D79009111217
:106B740059D7900910125C80700374FFF0E525600A
:106B8400559009191259CC125C7D700374FFF09072
:106B94000918E0FFD3648094804007A3E0700312D7
:106BA4005C87EF7003125B4190065AE0B4020C124A
:106BB4005D469009C17401F0E4801890065AE01211
:106BC4005D46B40109E49009C1F07D018037E49089
:106BD40009C1F0FD802F90091A1259CC125C7D7006
:106BE4000374FFF0900918E0FF7003125B41125C1C
:106BF400944009900919E07003125C87125D46E421
:086C04009009C1F0FD124EEEF3
:106C0C0090090CE4F0A37402F053F87FE59A20E7A6
:106C1C00FB90090CE0FEA3E02454F5827406125B91
:106C2C00BB0FBF00010EEF64324E70F590090DE002
:106C3C0024FFF090090CE034FFF0E0B4FFCBA3E0AC
:056C4C00B4FFC6D28771
:016C51002220
:10812000E4FD7C02900657E4F0A3DCFC7C007D02B9
:10813000E52F30E31C900658E0FFE52F5407FE744E
:1081400001A806088002C333D8FC4F900658F0807F
:1081500017900657E0FFAE2F7401A806088002C3EF
:1081600033D8FC4F900657F0C2A57C007D0153F830
:108170007FE59A20E7FB74572DF58274063C125B6D
:10818000BC0FBF00010EEF64324E70F5ED1D7001A3
:098190001CBCFFDABDFFD7D2A52B
:0181990022C3
:1080A200900731E0FFA3E0900721CFF0A3EFF0E5C6
:1080B200905440FF900731E4F0A3EFF09006FFE008
:1080C200FFA3E0900667CFF0A3EFF0E5905420FF06
:1080D2009006FFE4F0A3EFF0900721E07002A3E026
:1080E2007015900731E07002A3E0600B900721E465
:1080F200F0A304F0128D95900667E07002A3E07081
:108102001C9006FFE07002A3E06012900667E4F0A4
:0E811200A304F0900725124E32000000322226
:03500C00026658E1
:10665800C0E0C0F0C083C082C0D075D000C000C008
:0D66680001C002C003C004C005C006C00789
:10667500C28FAF231258A990093674011258C890D9
:10668500070CE0FF2402F582E43407F583E0900966
:1066950033F0EF14603E14606514607414700302E7
:1066A500673B1470030267692405600302678490E1
:1066B50006F1125A0E900939124E269009391258D0
:1066C50044FBD3124DA6402F900939124E320000DB
:1066D500FFFF80239006F3125A0E900939125A5C77
:1066E50090093912584BFBD3124DA6400A9009392F
:1066F500124E320000FFFF900939A3A380039006D4
:10670500F5E0FFA3E0900934CFF0A3EFF002678432
:106715009009361257F4F9124A77603F9006F8123D
:106725005B5F400474FF8001E4F0A3F0125C9440C9
:106735004E9006F880469009361257F4125CF560C3
:106745001A9006F9125B5F400474FF8001E4F0A320
:10675500F0125C9440299006F98021900934E4F008
:10676500A3F0801B9006F7125B5F400474FF800165
:10677500E4F0A3F0125C9440069006F7E014F0C232
:106785008653F87FE59A20E7FB900933E0F59BE413
:10679500FD0DEDB432FB900934E0FF7E0053F87F28
:1067A500E59A20E7FB8F9B7D000DEDB432FB900948
:1067B50034A3E0FF7E0053F87FE59A20E7FB8F9B2B
:1067C5007D000DEDB432FBD28690070CE004F0C3DA
:1067D50094064002E4F01280A290070BE024FA60D0
:1067E50009240670081278D2800312812090070BC5
:1067F500E004F0E05407F0125C31600764016003C7
:10680500026887125B2EC31259724006125AA20201
:0F68150068A012596C400302689412596C507CB1
:1068240090093DE4F09009361257F4F990000A12E9
:10683400591C24FE601014601C2402702B1259523F
:1068440064036024801C900710E0701C1259526489
:10685400036015800D900710E0600D125952640317
:10686400600690093D7401F090093DE0602E9004AB
:1068740004E0FF131313541F30E021127DBD125C9A
:016884003FD4
:10688500801912596C4003125AA212596C500C759A
:106895002E00752D00752C00752B00758DF0758BF0
:0168A50000F2
:1068A600D007D006D005D004D003D002D001D00046
:0B68B600D0D0D082D083D0F0D0E032F0
:068369009008FC124E26F4
:10836F00AF2EAE2DAD2CAC2B780F124DCA90090449
:10837F00124E2690090412584BFBC3E49BFFE49A5C
:10838F00FE740199FDE498FCA3124E269008FC128E
:10839F00589CFF90090812584BFB124C66C004C042
:1083AF0005C006C00790090012589CFFA312584B36
:1083BF00FB124C66D003D002D001D000EF2B125D20
:0683CF000E7810124DB7FC
:0183D5002285
:108683007C027D8F124B367C027D8F124B247C043F
:108693007D00124E959009E2124E269009E212587F
:1086A3009C125B159009E2125A5C9009E212584B36
:1086B300FBD3124DA6400A9009E2124E320000FF8E
:0786C300FF9009E2125BA425
:0186CA00228D
:10863500900A13EEF0A3EFF0C374469F74019E50A9
:108645003A900A13125A0E7BAA7AFEF9F8124D9047
:108655004029900A137C027D8F125964900A13EC0D
:10866500F0A3EDF0C3943CEC9400400CD3E0945897
:0E867500900A13E0940240037F01227F00224E
:0B76B2009009A8EEF0A3EFF0A3EDF0AC
:1076BD0014601E14602B14603814604524FE605154
:1076CD002406600302777B12595D9009A8EE0277BC
:1076DD007712595DEF2430FFEE34339009A802770D
:1076ED007712595DEF2460FFEE34669009A802779A
:1076FD007712595DEF2490FFEE34999009A8027727
:10770D007712595DEF24C0FFEE34CC9009A80277B3
:10771D0077AF03E4FCFDFE9009AB124E267BFF7A9A
:10772D00FF12587FFF7804124DB79009AB124E2609
:10773D007B297A0412587FFFE4FB7A04F9F8124C86
:10774D00F11258932400FFEE3408125B6F125A5950
:10775D009009AB12584BFBD3124DA6400A9009ABC2
:10776D00124E320000FFFF125BFCF0A3EFF0900908
:10777D00AAE0640660369009A8E0FEA3E0FF7C0451
:10778D007D00124E95125893125B15125A5990099D
:10779D00AB12584BFBD3124DA6400A9009AB124EBB
:1077AD00320000FFFF125BFCF0A3EFF09009A8E0A0
:0477BD00FEA3E0FF48
:0177C10022A5
:1072BA0042085F000042080A00004208050000C1B7
:0572CA0008C107C10628
:1085E600900805E475F001124B8BFCE5F064404CF5
:1085F60022D3900860E0940090085FE06480948045
:1086060022E0FEA3E0240CF582740822E0FBA3E03E
:10861600FAA3E0F98E8275830022900805F0A3F094
:0F86260022900801E004F022900800E004F02206
:0A8D8B00C207C208E4900809F022B4
:108B2100E490085FF0A3F090080AF0A3F0A3F0121C
:108B31008620900800F0A37440F0E4900808F02229
:068DA500128D8B028B21F0
:108C1F00E4F5848FC343C30175C04475CF8EC2C3BF
:098C2F0043E60290080704F0225C
:108CE500E4F58420C7FDC2C2128DA5E4900807F003
:018CF500225C
:0B8D6B00E4F584D2C290080704F02257
:0D8D4600AE07128C1F900804EFF0028DA5FF
:108A3000E4900A15F0A3F0300702FF222008FDD2CF
:108A400007900802E4F0A37410F090084DEFF0E4F2
:048A5000A3F07F010F
:018A540022FF
:1089000030070A900802E07002A3E070037F0022A3
:10891000900803E024FFF0900802E034FFF0900894
:108920004EE0FE04F0744F2EF582E43408F583EF38
:04893000F07F0122B1
:0B8D7600300707C207D208125021226C
:0E502100AF84E4F58420C7FDC2C4D2C58F84DD
:01502F00225E
:1082FA009009B0EBF0A3EAF0A3E9F0900807E07068
:10830A0002FF229009B3E0FE6005D3941040037F78
:08831A000022128A30EF6044DA
:10832200E49009B5F09009B3E0FF9009B5E0FEC30F
:108332009F501A9009B0128612124A90FF128900B9
:10834200EF7002FF229009B5E004F080D8E49008B3
:1083520009F0128D769009B4E070032008FD9008B0
:0483620009E0FF220D
:038366007FFF2274
:0E7C75009009E6EBF0A3EAF0A3E9F0A3EDF02E
:107C8300E4FF1285F750012253E6FD9008051286A2
:107C9300073EF583E0FF1285E67003128620128605
:107CA30027700312862EE4FE9009E9E0FDEEC39DE2
:107CB300502FEEC39F502A900805E0FC1286093C22
:107CC300F583E0FD9009E6128612ED124B02128550
:107CD300E67003128620128627700312862E0E800A
:107CE300C7EEC39F50131285E670031286201286D7
:107CF30027700312862E0E80E8900860E024FFF0C0
:107D030090085FE034FFF043E6029009E9E0FEEFFC
:087D1300C39E50028002AF067E
:017D1B002245
:0C8D5F001285F740047F0180027F002293
:03501800026F52D2
:106F5200C0E0C0F0C083C082C0D075D000C000C005
:036F620006C0075F
:106F6500C20DAFC1EF124E6F6F9B086F9B106FABD9
:106F7500186FB0206FBD286FEA306FF5386FFD6070
:106F85006FF8686FFD706FF8787005807005907008
:106F950075A00000708390084DE0F5C2C2C5900849
:106FA5004CE4F002708590084E802890080974FD25
:106FB500F0D2C4D2C502708590084EE0FF90084C0F
:106FC500E0C39F5014E0FF04F0744F2FF582E434C2
:106FD50008F583E0F5C2027085D2C4900809E4F093
:106FE500C208027085D2C590080974FEF00270854A
:106FF50002707AD2060270859007FFE4F002708570
:107005009007FFE07020E5C2F0E0FFC3900801E0C3
:107015009F7480F8900800E06480985003128B21DB
:107025009007FFE004F0900801E024FFF0900800CD
:10703500E034FFF090080A1286073EF583E5C2F0BA
:1070450090080AE475F001124B8BFEE5F064404EA2
:10705500700690080AF0A3F09007FFE014F0702086
:10706500900860E004F0701890085FE004F080106C
:1070750030060DC20690084CE4F0D2C58002D20D50
:10708500300D0EC2C6D2C6C2C5C2C4D2C2C20DC25E
:0370950008C2C36B
:10709800D007D006D000D0D0D082D083D0F0D0E0B6
:0170A80032B5
:058DAB00A2C7E433FF44
:018DB00022A0
:1084F200EFF0A3ECF0A3EDF0A3EBF0A3EAF0A3E915
:10850200F0227403F0A374E8F0A3E584F0E4F584A8
:1085120022D2C4D2C5D2C2C2C3E4900A1CF0FF2246
:10852200E0FBA3E475F001124BA1A9F0FA22E025C9
:10853200E044A0F5C27F032274FFF5F0124B8B4595
:02854200F02225
:068DB100C2C253E6FD22E0
:0677C20090091B1284F285
:1077C80090092412850420C7FDC2C4D2C2D2C5E4E0
:1077D800FF900A1CF030C3FDAEC1EE24F8602324EC
:1077E800F8601F24F8602924F8603024F8603424F5
:1077F800F8700302788524F8700302788D24380223
:107808007895EF700690091B128530C2C502789BE7
:1078180090091CE0F5C27F0502789B900A1C74034E
:10782800F08070EFB4050B90091CA3E0F5C27F0649
:107838008061EF64067034900923E090091E70059A
:107848001285228008E0FBA3E0FAA3E0F9124A7748
:10785800F5C2900922E024FFF0900921E034FFF0FE
:10786800E07002A3E0702C7F078028EFB40706D2EF
:10787800C47F09801E900A1C7405F08016900A1CAB
:107888007404F0800E900A1C7406F08006900A1C9E
:107898007401F0EFB40904C2C38025900A1CE0B457
:1078A800030B90092412853A6003128513900A1C71
:1078B800E06008C2C5D2C4C2C38005C2C30277DD76
:0978C80020C7FD900926E0F584BB
:0178D1002294
:0675880090093E1284F29E
:10758E0090094612850420C7FDD2C2C2C4D2C5E4FA
:10759E00FF900A1CF030C3FDAEC1EE124E6F75D1D6
:1075AE000075D40875D41075F918760420760C2859
:1075BE00762730762F38763740764750766F5800DC
:1075CE000075D1027675C2C5EF700990093E12851D
:1075DE003002767BEF6401600302767B90093EE019
:1075EE0025E044A1F5C27F0402767B90093FE0F5C9
:1075FE00C27F0502767B900A1C7403F0806FEFB495
:10760E00050B90093FA3E0F5C27F068060EFB4063C
:10761E0006D2C57F0180568018900A1C7404F08033
:10762E004C900A1C7406F08044EFB404047F028070
:10763E003C900A1C7405F08034900941128522E5B5
:10764E00C2124AF0900945E024FFF0900944E0345C
:10765E00FFF0E07002A3E07004C2C280107F0280CF
:10766E000CD2C47F098006900A1C7401F0EFB40995
:10767E0004C2C38025900A1CE0B4030B9009461285
:10768E00853A6003128513900A1CE06008C2C5D2C9
:10769E00C4C2C38005C2C30275A320C7FD900948AA
:0376AE00E0F58480
:0176B10022B6
:10732400900968EFF090096B1284FB900969ECF006
:03733400A3EDF0D6
:10733700753200543FF533543F6058C3744095335A
:10734700FFE49532FE90096EE0FCA3E0FDC39FECDD
:107357009E50068C308D3180048E308F3112742808
:1073670060037F022290096AE02531F0900969E005
:107377003530F0900970E0700B90096CE53085317D
:10738700F0124B8BC390096FE09531F090096EE0D6
:107397009530F090096EE0F530A3E0F531D3E53193
:1073A7009400E53094004076E5319440E530940050
:1073B700500F12742860037F0222E4F530F5318004
:1073C700DC900968E0FFA3E0FCA3E0FDA3E0FBA3DA
:1073D700E0FAA3E0F9900921E4F0A37440F09009E2
:1073E70070E0900923F01277C2900A1CE060037FD7
:1073F700022274C02531F53174FF3530F53090091C
:107407006AE02440F0900969E03400F0900970E0E8
:10741700708B90096C75F040124B8B0273A47F0040
:1074270022900968E0FFA3E0FCA3E0FDA3E0FBA333
:10743700E0FAA3E0F9900921E530F0A3E531F090F7
:0F7447000970E0900923F01277C2900A1CE0222E
:108C6A00900944E4F0A304F0127588900A1CE060AD
:078C7A00037F01227F0022AD
:108BD100900A1BEBF07B017A0A791B90096EE4F095
:0A8BE100A304F0E4A3F012732422B1
:108A9B00C007900980E0FFA3E0900944CFF0A3EF5B
:108AAB00F0D007127588900A1CE060037F01227FCB
:028ABB00002297
:108BEB00C007900988E0FFA3E090096ECFF0A3EFD8
:0A8BFB00F0E4A3F0D0071273242267
:108C05007B01E49009C7F0227422F0A3EFF0A322C0
:0A8C15007B01E49009C7F07D042202
:0E8713009009C3EBF0A3EAF0A3E9F0A3EDF0A8
:10872100E49009C8F09009C3E0FBA3E0FAA3E0F9E3
:10873100A3E09009B3F09009C7E09009B4F0E4FF19
:108741001282FAEFB4FF0D9009C8E0FE04F0EEC307
:06875100940340D17E00FC
:0187570022FF
:0B898E00900A10EBF0A3EAF0A3E9F060
:108999007E007F007D10124EC2900A10E0FBA3E01A
:1089A900FAA3E0F97D10127C75EF7002FF227F01B6
:0189B900229B
:10849A00900954128C0D7413F0124A77900957F010
:1084AA00900001124A90900958F0900002124A90E6
:1084BA00900959F0900003124A9090095AF09000DE
:1084CA0004124A9090095BF0900005124A909009B4
:1084DA005CF0900006124A9090095DF07A0979548E
:0884EA00128C057D0A028713C4
:108C38009009EA128C0D7403F0A374FFF07A097995
:098C4800EA128C057D0402871379
:108C81009009EE128C0D741CF0A374FFF07A09792F
:078C9100EE128C150287139F
:108C5100E49009F2F0A3EFF0A3740AF0A3EFF07A25
:098C61000979F2128C1502871347
:108B4100E0FEA3E0A60608F6E4F584C2AF43B70150
:0F8B510022E475F001024BA1EEF0A3EFF0A32296
:10889500AB84A2AF920EE4FCFDED9009F6124E26D4
:1088A5009009F8781E128B41438F02438F0118E619
:1088B500FE08E6F5828E83E4F053B7FEF58FA20E2F
:0688C50092AFAF038F84A7
:0188CB00228A
:02879C00AB052B
:10879E00AA84A2AF920FE4FCFDED9009FA124E26C8
:1087AE00EBFF3395E0FEEFF44E601C9009FC78343D
:1087BE00128B41758F0118E6FC08E6F5828C83EB6F
:0F87CE00F053B7FEE4F58FA20F92AFAF028F8486
:0187DD002279
:10843C009009C9128B59ECF0A3EDF0A3EAF0A3EB71
:10844C00F09009CDE07002A3E060429009C9E0FE13
:10845C00A3E0FFA3E0FCA3E0F5828C83E0FD128790
:10846C009C9009CEE024FFF09009CDE034FFF09011
:10847C0009CCE004F070069009CBE004F09009CA36
:0E848C00E004F070BC9009C9E004F080B42256
:088D9D00E4900000F0A3F022B5
:108A0A00900000E0FEA3E0FF128895900000E0FECF
:108A1A00A3E0FF7C007D027B007A0412843CE49090
:068A2A000000F0A3F022A1
:0A802100A9059009CFEEF0A3EFF0DF
:10802B00EE54FCFE900000E0FCA3E0FD7002EE6C51
:10803B00604CED4C6003128A0A9009CFE0FEEE54BF
:10804B00FCFE7F00900000F0A3EFF09009D1128BA3
:10805B00597400F0A37402F07E049009D1128B5274
:10806B0085F082F583E493FD9009D3128B5285F052
:10807B0082F583EDF0EF1F70011EEF4E70DC90095F
:10808B00CFE0FCA3E0FDEC5403FC74022DF58274ED
:06809B00003CF583E9F052
:0180A10022BC
:10881F009009B6128B59EBF0A3EAF0A3E9F0900997
:10882F00BB74FFF5F0124BA145F0601E9009B61214
:10883F008B52AFF0FE9009B8E0FBA3128B52A9F058
:0B884F00FA124A77FD12802180D4222B
:10821200E47F01FEFDFCE0F8A3E0F9A3E0FAA3E0AD
:10822200FB221287589008F0124E269008E9E025AA
:10823200E02499F582E43407F583E0FEA3E022FB13
:10824200C374FF9BFF740F9EFEE49400FDE4940050
:10825200FC229008E8E075F002A42405F582E5F01E
:108262003404229008E9E025E02433F582E434075F
:1082720022E47BFF7A0FF9F822E0FCA3E0FDA3E001
:05828200FEA3E0FF2255
:086DE2009008E8EFF0A3EDF0CA
:106DEA0012826912823AFBAA0612822DFFC3EF9B16
:106DFA00FFEE9A12824A9008EC124E26E49008EAB4
:106E0A00F0A3F07F0FFEFDFCA3128218C3124D906F
:106E1A0040089008EAE4F0A304F074FF7FF1FEFD55
:106E2A00FC9008EC128218D3124D90500874FF900F
:106E3A0008EAF0A3F09008EAE0FEA3E0FF4E700330
:0B6E4A00026F51EFF47002EEF4706173
:106E550012826512823AFFE4FCFD9008F8124E2674
:106E65009008F8128212C3124D90500A9008F81239
:106E75004E320000000112825412823AFFE4FCFDFA
:106E8500128274124C669008F8128218128224FF3E
:106E9500E4FCFD9008F0128218124C669008F4127A
:0E6EA5004E261282739008F412827B128758D8
:0F6EB300026F249008EAE07004A3E06401706F9E
:106EC20012825412823A128241128273124C6690DA
:106ED20008F0124E2612826512823A1282419008FE
:106EE200F4124E269008F4128212C3124D90500AE8
:106EF2009008F4124E32000000019008F012827BDA
:106F0200A31282181282241282419008F01282186F
:106F1200124C66128273128758C374FF9FFF740F5C
:0F6F22009EFE128254F583EEF0A3EFF012893435
:106F31009008E9E0FF25E02499F582E43407F58320
:106F4100E0FCA3E0FDEF128269F583ECF0A3EDF024
:016F5100221D
:108D16000001FF00FF000001010000FF00FF01004D
:1072CF00040800000000041A00000000041600006B
:1072DF00000002130000011500010D00020E000056
:1072EF0003100000004408B4000000004408AC0084
:1072FF000000004208B200004108B0004108B10090
:1083D600AF0BAE0AAD09AC08024D839008B4E0FCC1
:1083E600A3E0FDA3E0FEA3E0FFEC4D4E4F22900973
:1083F6008AA3A3E0FEA3EE2290098AA3A3A3E02208
:10840600FFE4FEFDFCEF22AFB0FEEF5407FFE47879
:1084160010024DDEEF4BFFEE4AFEED49FDEC482221
:108426009009FFE0FBA3E0FAA3E0F92290098AA3F2
:06843600E0FDA3A3ED220E
:1086CB00D2B3C2B4128ABDE4FCFDC004C005C0061F
:1086DB00C00712840DD003D002D001D00012841A2F
:1086EB008F198E188D17F5168F1D8E1C8D1BF51A75
:1086FB00AF907513008F147B017A0879B88B108AB1
:08870B001189128A0E890F2268
:058287009009FEEFF07C
:10828C00E50F2401FFE4350EFAA907A37401F0A34E
:10829C00EAF0A3E9F012842674019008CC6B700804
:1082AC00E965827003EA6583700D9009FF04F0A301
:1082BC007408F0A374B8F0128426E5108511838538
:1082CC0012826B7008E965827003EA6583601E9008
:1082DC0009FEE0850F82850E83F09009FFA3E0FA7A
:0D82EC00A3E0AE028E0EF50F9009FEE0F04B
:0182F9002262
:1085440053E6F7E5108511838512826401700AE50C
:108554000F65827004E50E65837003FF802FAB10F6
:108564000512E512AA117002051114F9124A77FFD7
:1085740074019008CC6B700AE51265827004E511F1
:10858400658370097510017511087512B843E60802
:0185940022C4
:03501E0002627CAF
:10627C00C0E0C0F0C083C082C0D075D000C000C0E8
:10628C0001C002C003C004C005C006C00720DF0364
:03629C000265CCCC
:10629F00E50C6005D50C02D210128ABDE4FCFDC0DE
:1062AF0004C005C006C00712840DD003D002D00170
:1062BF00D00012841A8F0B8E0A8D09F508AF1DAE10
:1062CF001CAD1BAC1AAB0BAA0AA909F8C3124DA639
:1062DF006031E50B651DFFE50A651CFEE509651BD1
:1062EF00FDE508651AFC90098A124E2690098A125C
:1062FF0083E46003751503850B1D850A1C85091B37
:10630F0085081AE51570030265201515E51560035C
:10631F00026520E519650BFFE518650AFEE51765AF
:10632F0009FDE5166508FC90098A124E261283FEB8
:10633F005401FFEF60101283D6EF540112840660F0
:10634F00057F011282871283FE5402FFEF60101245
:10635F0083D6EF540212840660057F0212828712E1
:10636F0083FE5404FFEF60101283D6EF540412849F
:10637F000660057F031282871283FE5408FFEF60C9
:10638F00101283D6EF540812840660057F04128220
:10639F00871283FE5410FFEF60101283D6EF541054
:1063AF0012840660057F051282871283FE5420FF38
:1063BF00EF60101283D6EF542012840660057F061B
:1063CF001282871283FE5440FFEF60101283D6EFC4
:1063DF00544012840660057F071282871283FE5491
:1063EF0080FFEF60101283D6EF5480128406600591
:1063FF007F081282871283F45401FEEE601212831B
:10640F00D6EE5401FEE4FDFCEE60057F0912828793
:10641F001283F45402FEEE60121283D6EE5402FE83
:10642F00E4FDFCEE60057F0A1282871283F45404A8
:10643F00FEEE60121283D6EE5404FEE4FDFCEE6015
:10644F00057F0B1282871283F45408FEEE6012123E
:10645F0083D6EE5408FEE4FDFCEE60057F0C12823D
:10646F00871283F45410FEEE60121283D6EE54108E
:10647F00FEE4FDFCEE60057F0D1282871283F4545B
:10648F0020FEEE60121283D6EE5420FEE4FDFCEEE9
:10649F0060057F0E1282871283F45440FEEE601265
:1064AF001283D6EE5440FEE4FDFCEE60057F0F1222
:1064BF0082871283F45480FEEE60121283D6EE545C
:1064CF0080FEE4FDFCEE60057F101282871284329D
:1064DF005401FDED60131283D6E4FEED5401FDE48B
:1064EF00FCED60057F111282871284325404FDED9A
:1064FF0060131283D6E4FEED5404FDE4FCED600559
:10650F007F13128287850B19850A1885091785084D
:10651F0016C2DF1283D690098E124E269008B4E071
:10652F00FCA3E0FDA3E0FEA3E0FF9008AC124E2613
:10653F0090098EA3E0FDE4FFFEED5402FDE4FC9014
:10654F0008B4124E261283E160409008AC1283E427
:10655F0070069008B2F0A3F09008B3E004F0700654
:10656F009008B2E004F0D39008B3E094589008B2CA
:10657F00E06480948240469008B1E070057F161267
:10658F0082879008B17401F080331283E1702E90EE
:10659F0008AC1283E460269008B2E0FEA3E0FFD3BC
:1065AF00940AEE64809480400FEF9458EE648094C8
:0D65BF008250057F121282879008B1E4F02F
:0A65CC009008B0E004F0640270676C
:1065D600E590540390098AF0E0FDFFE5146F54033B
:1065E6006050E514AE137802C333CE33CED8F97EAD
:1065F60000540CFFED5403FDEF4D2416F582EE34E6
:106606008DF583E493FF90098BF0A3E50DF0EF255C
:106616000DF50DE0650D30E11090098BE0B4010435
:106626007F1480027F1512828790098AE075130015
:07663600F5149008B0E4F038
:10663D00D007D006D005D004D003D002D001D000B1
:0B664D00D0D0D082D083D0F0D0E0325B
:108ABD00D2B4E4FBC2B3ED25E0FDEC33FC30B504DC
:108ACD00ED4401FDD2B30BEBB410E9C2B4AF05AE6A
:018ADD000494
:018ADE002275
:10730F0041099200C10AC10947099318100C0806D8
:02731F00040365
:108A7800900474E0C3135403FF2290000A124A9032
:108A88001313135407FF22900A02E0FBA3E0FAA392
:038A9800E0F922E0
:108B0000900003124A902406600D14601014600A4D
:108B10002404700C027456028B7F028D26128D364F
:018B20002232
:108B7F00D20AE4900992F0128A78BF030E9004048F
:0C8B8F00E04408F0E4FF1288CCD2092278
:108D2600C20A128A78BF0307900404E054F7F022BF
:108D3600D20A128A78BF0307900404E04408F0229E
:10745600AF23EF3395E0FE7C007D0B124B24746B5B
:107466002FF974043EFA900A027401F0A3EAF0A31D
:10747600E9F0200A03027587900992E0FF04F0EF15
:10748600B460037401F0128A8F900009124A90C307
:0A74960013540364036003027587BA
:1074A000AF23EF3395E0FEEF25E0FFEE33FE7445AA
:1074B0002FF58274043EF583E0FEA3E0FFD3945BD6
:1074C000EE940F4007E4900A05F08058D3EF94172C
:1074D000EE940C4008900A057401F08047D3EF94B5
:1074E000EBEE94084008900A057402F08036D3EF62
:1074F00094A7EE94064008900A057403F08025D303
:10750000EF94FFEE94024008900A057404F0801492
:10751000D3EF9416EE9401900A0540057405F080AF
:10752000037406F0900992E024FFFFE434FFFE901C
:107530000A05E02493F582E43409F583E0FD3395F0
:10754000E0FC124B36ED703F300903C20922900473
:1075500004E0131313541F30E02D128A8F128A8215
:1075600064016015BF0206900710E0600C128A8269
:10757000BF0314900710E0600E127DBD74FFF52E5E
:07758000F52DF52C752B7FA2
:0175870022E1
:02732100C10B9E
:107BC000900950E0FF75F018A42402F582E5F03426
:107BD000A4F583EF2583AF8222124AF0900A07E0D2
:107BE000FBA3E0FAA3E022FE7A0479037B0190096B
:107BF000BB7401F0A37418F022AFF0FEE0FCA3E028
:107C0000F5828C83E493FD2290094CF0A3EFF0E41D
:107C1000900952F0A3F02275F018EEA42402F58228
:107C2000E5F034A4F583EE2583AF8222F9E43AFA35
:107C3000024A777E007C017D18124B2474022FF9D2
:107C400074A43EFA22EFF0A3EDF0A3EBF0A2AFE4B0
:107C500033A3F0C2AF22E475F001024BA1900953A7
:107C6000E004F022900952E004F022FDEDFFEEF076
:057C7000A3EFF0E42287
:10893400300027200B263002237F407E0D7D037CF0
:1089440000900633E0F8A3E0F9A3E0FAA3E0FBC348
:0D895400124DA67002D203D20B22D20422D3
:05896100900A17EFF081
:10896600128D9DE4900A18F0900A17E0FFA3E0FE2E
:10897600C39F5011127C17127BE712881F900A18AA
:08898600E004F080E3028A0A1C
:10885A00900A197402F0E4A3F0128D9D7EA47F00A1
:10886A007A0A79191288877EC47FD27A0A791A120B
:0D887A008887128A0A1279E17F1E02896147
:0E8887007B019009BBE4F0A304F012881F22CD
:108B6000E5B030E01190C4D2E493F4600990A40021
:0F8B7000E4936402600312885AE4900402F02236
:10859500C20B900402E0FFC3941E503A127C337B59
:1085A500FF78037C047D017E017F18124A2FE4FFCA
:1085B50075F00BEFA42473F582E5F03404F583E040
:1085C500C4135401FE74112FF582E43407F583EECC
:1085D500F00FEFB410DA900633124E3200000000AF
:0185E5002273
:108B9B00900402E0C3941E5012128D9D9004021299
:0C8BAB007BC3127BE712881F128A0A228B
:068DB700128B9BC20B228F
:087D1C00900928EDF0A3EBF043
:107D2400A3E004F090092DEFF0A3EBF0900928E014
:107D3400FF90092DE0FED39F5068127C1790092F05
:107D4400F0A3EFF090092E127BC3900931F0A3EF5A
:107D5400F0E490092BF0A3F0900931127C569009BD
:107D64002F127BF9128021900930E004F070069004
:107D7400092FE004F090092CE004F0700690092B20
:107D8400E004F0C390092CE0941890092BE09401CE
:107D940040C6128A0A90092DE004F0A3E004F00220
:107DA4007D30900402E0FF900929E0D39F5009A39D
:087DB400E0C39F400312859516
:017DBC0022A4
:0F70A90090094AEDF0900949EFF090094BEBF098
:1070B800900950EFF0A3EBF090094AE0FF900950D7
:1070C800E0D39F40030271A3A3127BC3127C0890F4
:1070D8000952E0FEA3E0FFC39418EE9401502A90F1
:1070E800094C127BFC741B2FF58274053EF583ED69
:1070F800F090094DE004F0700690094CE004F0129D
:107108007C5D70CB127C6480C6127BC090094EF007
:10711800A3EFF0900951127BC3127C0890094C121E
:107128007C5690094E127BF912802190094FE00499
:10713800F0700690094EE004F0127C5D7003127C3A
:1071480064C3900953E09418900952E0940140CC2C
:10715800127BC090094E127C0B900952E0FCA3E010
:10716800FDC39418EC9401502290094E127C56AF3E
:10717800F0FE741B2DF58274053CF583E0FD12804A
:1071880021127C5D70D3127C6480CE128A0A900929
:1071980050E004F0A3E004F00270C0900402E0FFA5
:1071A80090094BE0FED39F5020900949E0FDA3E0F1
:1071B800C39DFDE49400FCEE7A002DFDEA3CFCC37F
:1071C800ED9F7480F86C985013900402E0FF9009CA
:0F71D80049E0D39F5009A3E0C39F400312859560
:0171E7002285
:037F910090095EF6
:107F9400127C45128DB190095FE0FE90095EE0907D
:107FA4000966127C6B900962F0900960E0FF900909
:107FB40066E0FCA3E0FD7B017A05791B9009801241
:107FC4007BF1128A9B900967E02418F0900966E01F
:107FD4003401F0900962E0FF127C33A374FFF0A334
:107FE400EAF0A3E9F0128D9D900963A3E0FAA3E0FF
:107FF400AE02FF7A05791B127BEC12881F128A0AE3
:10800400900962E004F0E0C3941E409D900724E0D0
:0C801400FF128D46900961E024FF92AF3E
:01802000223D
:03819A00900971D8
:10819D00127C45128DB1900972E0FE900971E0904C
:1081AD000976127C6B900975F0900975E0FFC39408
:1081BD001E504175F018EF127BC8FE900978F0FA49
:1081CD00A3EFF0FB900973E0FF900976E0FCA3E0CC
:1081DD00FDA9037BFF900988127BF1128BEB9009AF
:1081ED0077E02418F0900976E03401F0900975E0FD
:1081FD0004F080B5900724E0FF128D46900974E0DD
:04820D0024FF92AF09
:01821100224A
:1079E100E4900403F0A3E054F8F054F7F0E4900AB3
:1079F10006F0900A06E0FFC39433501B75F002EFC6
:107A0100A42405F582E5F03404F583E4F0A3F090B5
:107A11000A06E004F080DB9004657408F0A3E4F04A
:107A2100900A06F0900A06E0FFC394104003027A20
:017A3100E173
:107A3200EF75F00BA4246BF9740435F0FAA374010A
:107A4200F0A3EAF0A3E9F0127BDCF9E4127BD9F9A6
:107A5200900001E4124B02900002E4F5F0124C395E
:107A6200900004E4124B02900005E4124B02E92458
:107A720006127C2C54C0127BD92407127C2C54F899
:107A8200124AF054C7127BD92408127C2C54F812E3
:107A92004AF054F7124AF054EF124AF054DF124AF5
:107AA200F054BF124AF0547F127BD92409127C2C65
:107AB20054FE124AF054F94402124AF054C74428C0
:107AC200127BD9240A127C2C54F84405124AF05431
:067AD200C74408124AF04F
:097AD800900A06E004F0027A2590
:017AE1002282
:03000000024000BB
:03000300025003A5
:03000B000250069A
:030013000250098F
:03001B0002500C84
:0300230002500F79
:03002B000250126E
:0300330002501563
:03003B0002501858
:0300430002501B4D
:03004B0002501E42
:0300530002502137
:03005B000250242C
:0300630002502721
:03006B0002502A16
:0300730002502D0B
:03007B0002503000
:03008300025033F5
:03008B00025036EA
:03009300025039DF
:03009B0002503CD4
:0300A30002503FC9
:10400000787FE4F6D8FD9000007F007E20E4F0A3E6
:0A401000DFFCDEFA75813502405531
:10401A0002503CE493A3F8E493A34003F68001F230
:10402A0008DFF48029E493A3F85407240CC8C333A7
:10403A00C4540F4420C8834004F456800146F6DF76
:10404A00E4800B01020408102040809071E8E47EAD
:10405A00019360BCA3FF543F30E509541FFEE4936B
:10406A00A360010ECF54C025E060A840B8E493A332
:10407A00FAE493A3F8E493A3C8C582C8CAC583CA5D
:10408A00F0A3C8C582C8CAC583CADFE9DEE780BE15
:017323000069
:10495F00E709F608DFFA8046E709F208DFFA803E3A
:10496F0088828C83E709F0A3DFFA8032E309F60827
:10497F00DFFA8078E309F208DFFA807088828C838F
:10498F00E309F0A3DFFA806489828A83E0A3F60843
:10499F00DFFA805889828A83E0A3F208DFFA804C1D
:1049AF0080D280FA80C680D4806980F280338010F4
:1049BF0080A680EA809A80A880DA80E280CA80335D
:1049CF0089828A83ECFAE493A3C8C582C8CCC583D5
:1049DF00CCF0A3C8C582C8CCC583CCDFE9DEE780A5
:1049EF000D89828A83E493A3F608DFF9ECFAA9F024
:1049FF00EDFB2289828A83ECFAE0A3C8C582C8CC7A
:104A0F00C583CCF0A3C8C582C8CCC583CCDFEADE92
:104A1F00E880DB89828A83E493A3F208DFF980CCF4
:104A2F0088F0EF60010E4E60C388F0ED2402B404ED
:104A3F000050B9F582EB2402B4040050AF23234594
:064A4F0082239049AF73C1
:104A5500C2D530F707B2D563F0FF05F030E70CB2E9
:104A6500D5F4048463F0FF05F080018430D502F4A9
:024A7500042219
:104A7700BB010689828A83E0225002E722BBFE023D
:094A8700E32289828A83E4932270
:104A9000BB010CE58229F582E5833AF583E02250DB
:104AA00006E92582F8E622BBFE06E92582F8E22225
:0D4AB000E58229F582E5833AF583E493223F
:104ABD00BB010FF8E58229F582E5833AF583E028FD
:104ACD00F0225009C58229F8E58226F622BBFE099F
:104ADD00C58229F8E22582F222F8EA2583F583E9D9
:034AED00932822E9
:104AF000BB010689828A83F0225002F722BBFE01A5
:024B0000F3229E
:104B0200F8BB010DE58229F582E5833AF583E8F0E9
:104B1200225006E92582C8F622BBFE05E92582C895
:024B2200F2227D
:104B2400EF8DF0A4A8F0CF8CF0A428CE8DF0A42EA5
:024B3400FE225F
:104B3600BC000BBE0029EF8DF084FFADF022E4CC63
:104B4600F875F008EF2FFFEE33FEEC33FCEE9DEC2C
:104B5600984005FCEE9DFE0FD5F0E9E4CEFD22ED72
:104B6600F8F5F0EE8420D21CFEADF075F008EF2FBC
:104B7600FFED33FD4007985006D5F0F222C398FDAD
:054B86000FD5F0EA224A
:104B8B00C5F0F8A3E028F0C5F0F8E58215827002B5
:064B9B001583E038F02252
:104BA100A3F8E0C5F025F0F0E582158270021583C7
:064BB100E0C838F0E82224
:104BB700BB010A89828A83E0F5F0A3E022500687C9
:104BC700F009E71922BBFE07E3F5F009E31922898B
:0B4BD700828A83E493F5F074019322BE
:104BE200BB0110E58229F582E5833AF583E0F5F011
:104BF200A3E0225009E92582F886F008E622BBFEEE
:104C02000AE92582F8E2F5F008E222E5832AF58333
:084C1200E993F5F0A3E99322F8
:104C1A00BB010A89828A83F0E5F0A3F0225006F7E5
:0F4C2A0009A7F01922BBFE06F3E5F009F31922E2
:104C3900F8BB0111E58229F582E5833AF583E8F0AD
:104C4900E5F0A3F0225009E92582C8F608A6F0226A
:0D4C5900BBFE09E92582C8F2E5F008F22251
:104C6600E88FF0A4CC8BF0A42CFCE98EF0A42CFCED
:104C76008AF0EDA42CFCEA8EF0A4CDA8F08BF0A46B
:104C86002DCC3825F0FDE98FF0A42CCD35F0FCEBCA
:104C96008EF0A4FEA9F0EB8FF0A4CFC5F02ECD398F
:0F4CA600FEE43CFCEAA42DCE35F0FDE43CFC22FC
:104CB50075F008758200EF2FFFEE33FECD33CDCCB6
:104CC50033CCC58233C5829BED9AEC99E582984039
:104CD5000CF582EE9BFEED9AFDEC99FC0FD5F0D616
:104CE500E4CEFBE4CDFAE4CCF9A88222B800C1B940
:104CF5000059BA002DEC8BF084CFCECDFCE5F0CB7E
:104D0500F97818EF2FFFEE33FEED33FDEC33FCEBB6
:104D150033FB10D703994004EB99FB0FD8E5E4F971
:104D2500FA227818EF2FFFEE33FEED33FDEC33FC5E
:104D3500C933C910D7059BE99A4007EC9BFCE99A52
:104D4500F90FD8E0E4C9FAE4CCFB2275F010EF2F97
:104D5500FFEE33FEED33FDCC33CCC833C810D70797
:104D65009BEC9AE899400AED9BFDEC9AFCE899F8D2
:0E4D75000FD5F0DAE4CDFBE4CCFAE4C8F92265
:10875800C2D5E830E70FB2D5E4C39BFBE49AFAE44C
:1087680099F9E498F8EC30E717B2D512878E124CD5
:10877800F1E4C39BFBE49AFAE499F9E498F88003DE
:10878800124CF130D50DE4C39FFFE49EFEE49DFD3D
:04879800E49CFC223F
:0D4D8300CFF4CFCEF4CECDF4CDCCF4CC22C5
:104D9000EB9FF5F0EA9E42F0E99D42F0EC6480C89A
:064DA00064809845F0223A
:104DA600EB9FF5F0EA9E42F0E99D42F0E89C45F063
:014DB60022DA
:104DB700E8600FECC313FCED13FDEE13FEEF13FFDA
:034DC700D8F122FE
:104DCA00E86010ECA2E713FCED13FDEE13FEEF13FF
:044DDA00FFD8F022EC
:104DDE00E8600FEFC333FFEE33FEED33FDEC33FC33
:034DEE00D8F122D7
:104DF1007401FF3395E0FEFDFCA3A3A3E0CF2FF0E8
:104E0100E582158270021583E0CE3EF0E5821582BF
:104E110070021583E0CD3DF0E582158270021583A5
:054E2100E0CC3CF02292
:0C4E2600ECF0A3EDF0A3EEF0A3EFF022FF
:104E3200A8828583F0D083D082124E49124E491245
:104E42004E49124E49E473E493A3C583C5F0C5836A
:104E5200C8C582C8F0A3C583C5F0C583C8C582C8CA
:014E6200222D
:0C4E6300A42582F582E5F03583F583225A
:104E6F00D083D082F8E4937012740193700DA3A3D2
:104E7F0093F8740193F5828883E4737402936860E6
:064E8F00EFA3A3A380DFE6
:104E9500EC8EF0A4CCC5F0CCCDF8EFA4CEC5F02DAA
:104EA500FDE43CFCE8A42EC8C5F03DFDE43CFCEF68
:0D4EB500A4FFE5F028FEE43DFDE43CFC22F6
:104EC200EF4E6012EF60010EEDBB010B89828A8307
:104ED200F0A3DFFCDEFA2289F05007F709DFFCA914
:0C4EE200F022BBFEFCF309DFFCA9F0226B
:00000001FF
